:100000000C942A001895000018950000189500001F
:10001000189500001895000018950000189500002C
:10002000189500001895000018950000189500001C
:10003000189500000C948E070C94C00718950000CA
:1000400018950000189500001895000018950000FC
:10005000189500008FE58DBFC0E4E6E24E2E88E0E3
:100060008EBFD8E0F8E05F2EEEEFF7E0A0E6B0E05C
:10007000A89584B7082E877F84BF88E1992781BD22
:1000800091BD88278D933197E9F786E089B980E0A3
:1000900080BD88E18AB96624579A84B7877F84BF78
:1000A0008DE181BD85E081BD8D988E988F98789483
:1000B0000E94AD08A4E7B1E0E4E6F1E10E94D705B3
:1000C000A6E7B1E0E6E6F1E10E94D705A8E7B1E0D6
:1000D000E8E6F1E10E94D705ACE7B1E0ECE6F1E13A
:1000E0000E94D705A0E8B1E0E0E7F1E10E94D70562
:1000F000A4E8B1E0E4E7F1E10E94D705A8E8B1E0A7
:10010000E8E7F1E10E94D705ACE8B1E0ECE7F1E106
:100110000E94D705A0E9B1E0E0E8F1E10E94D7052F
:10012000A4E9B1E0E4E8F1E10E94D705A8E9B1E073
:10013000E8E8F1E10E94D705ACE9B1E0ECE8F1E1D3
:100140000E94D705A0EAB1E0E0E9F1E10E94D705FD
:10015000A4EAB1E0E4E9F1E10E94D705A8EAB1E040
:10016000E8E9F1E10E94D705ACEAB1E0ECE9F1E1A0
:100170000E94D705A0EBB1E0E0EAF1E10E94D705CB
:10018000A4EBB1E0E4EAF1E10E94D705A8EBB1E00D
:10019000E8EAF1E10E94D705ACEBB1E0ECEAF1E16D
:1001A0000E94D705A0ECB1E0E0EBF1E10E94D70599
:1001B000A4ECB1E0E4EBF1E10E94D705A8ECB1E0DA
:1001C000E8EBF1E10E94D705ACECB1E0ECEBF1E13A
:1001D0000E94D705A0EDB1E0E0ECF1E10E94D70567
:1001E000A4EDB1E0E4ECF1E10E94D705A8EDB1E0A7
:1001F000E8ECF1E10E94D70589EF8093DC018FEFF5
:100200008093DD018EEF8093DE0180E08093DF013B
:1002100084E68093E00188EC8093E10182E380939F
:10022000E2018EE18093E30188E28093E40180E5BE
:100230008093E5018FE58093E60186E98093E701ED
:1002400080EF8093E80187EF8093E90188EF809346
:10025000EA0186EE8093EB0187EE8093EC0188EE55
:100260008093ED0189EE8093EE018FEE8093EF0194
:1002700086EF8093F0018AEF8093F1018BEF8093FA
:10028000F2018CEF8093F30180E08093F401A0E30E
:10029000B0E08C9185FBABE6B1E08C9180F98C935A
:1002A000A0E3B0E08C9186FBABE6B1E08C9181F9E4
:1002B0008C93A0E3B0E08C9187FBABE6B1E08C912E
:1002C00082F98C930027A9E6B1E08C9187FB0EF4AC
:1002D00001E041E0041711F00C949E018091690146
:1002E0008F7780936901A4EEB0E03FE30E946A0437
:1002F000A4EEB0E08C91082F0A3011F00C949C0110
:10030000A4EEB0E00E949308082F41E0041BAAE687
:10031000B1E00C93A4EEB0E00E949308EA2FFB2F0B
:1003200000916A013197E01BF10B0FEFA4EEB0E0F2
:100330000E948B080C9478010E94AE01A8950C9441
:100340006201A4EEB0E00E94A9040E94B6040895E0
:10035000809169018068809369010895A4EEB0E0FE
:100360008C91082F033211F00C94BA010E94A10164
:100370000C942F02A4EEB0E0E4E6F1E12FEF91E05F
:100380000E94E205A3E7B1E00C93009173010030F5
:1003900018F011F00C94CE010C941D02A4EEB0E004
:1003A000ECECF1E12FEF91E00E94E205002F00302C
:1003B00080E010F009F081E08F9340917301A4EE8A
:1003C000B0E0ECECF1E12FEF91E00E94E205002FAC
:1003D000041781E008F080E09F918923882311F4BD
:1003E0000C94FA010E94A1010E9430020C942F0289
:1003F0000C941B02E4EEF0E000917301A4E2B1E082
:100400000E948B08A4E2B1E00E945308ACE6B1E080
:100410000C9340916B0100916C01041711F00C9446
:1004200017020E9430020C942F020C941B020E94AF
:10043000A1010C942F020C942F0240916B010091AA
:100440006C01041711F00C942B020E9430020C94E2
:100450002F020C942F020E94A1010C942F020895E8
:1004600081E08093F601A4E2B1E088278C93A4E6B2
:10047000B1E088278C93AFE6B1E0E0E6F1E10E94BD
:100480007A0780E090E0ADE6B1E08D939C93A4EE16
:10049000B0E00E949308082F0F93A4EEB0E0E4E7C9
:1004A000F1E0222791E00E94E205402F0F91041B0A
:1004B000A3E7B1E00C93A4EEB0E00E949308EA2F0A
:1004C000FB2F009173013197E01BF10B0FEFA4E2BA
:1004D000B1E00E948B0881E08093F5010091F50165
:1004E000043018F011F00C94E90281E4482FA5EFD4
:1004F000B1E0AD90BB24A3E2B1E0AA0DBB1D0C910D
:10050000041781E008F480E08F938AE5482FA5EF77
:10051000B1E0AD90BB24A3E2B1E0AA0DBB1D0C91EC
:10052000041781E010F009F080E09F9189238F93F8
:1005300081E6482FA5EFB1E0AD90BB24A3E2B1E086
:10054000AA0DBB1D0C91041781E008F480E09F9177
:10055000892B8F938AE7482FA5EFB1E0AD90BB249C
:10056000A3E2B1E0AA0DBB1D0C91041781E010F0CD
:1005700009F080E09F918923882311F40C94E10213
:10058000A5EFB1E0AD90BB24A3E2B1E0AA0DBB1D85
:100590008C91A6EFB1E0AD90BB24A3E6B1E0AA0D2B
:1005A000BB1D8C93A6EFB1E08C918F5F8C9380E0A4
:1005B000A6EFB1E0AD90BB24A3E6B1E0AA0DBB1D50
:1005C0008C93A5EFB1E08C918F5F8C9310F40C9419
:1005D0006E02A4E6B1E00E949308082F033011F0E8
:1005E0000C942D03E4E6F1E0A4E6B1E00E9482075A
:1005F00080E08093F5010091F501093118F011F0C8
:100600000C942D03E5EFF1E00191112744E050E057
:100610000E94CD05E4E7F1E0E00FF11FA4E6B1E0B0
:100620000E949B0811F00C942503A5EFB1E0AD905A
:10063000BB24ABEDB1E0AA0DBB1D8C91ADE6B1E0E2
:100640008D9388278C930C942D03A5EFB1E08C91AA
:100650008F5F8C9310F40C94FB0281E08093F60181
:10066000A4E6B1E088278C93A4E2B1E0E6E7F1E0EC
:10067000222791E00E94E205A3E7B1E00C930091EC
:100680007301003011F00C944C03A4E2B1E00E941D
:100690009308A3E7B1E08C9381E08093F50140914A
:1006A00073010091F501041718F011F00C94A703E1
:1006B00080E3482FA5EFB1E0AD90BB24A3E2B1E009
:1006C000AA0DBB1D0C91041781E008F480E08F9304
:1006D00089E3482FA5EFB1E0AD90BB24A3E2B1E0E0
:1006E000AA0DBB1D0C91041781E010F009F080E009
:1006F0009F918923882311F40C949F03A5EFB1E007
:10070000AD90BB24A3E2B1E0AA0DBB1D8C91A6EF76
:10071000B1E0AD90BB24A3E6B1E0AA0DBB1D8C9364
:10072000A6EFB1E08C918F5F8C9380E0A6EFB1E0F3
:10073000AD90BB24A3E6B1E0AA0DBB1D8C93A5EF41
:10074000B1E08C918F5F8C9310F40C944F03ADE665
:10075000B1E00D911C910F931F93A4E6B1E00E94AC
:100760005308402F512F1F910F91040F151FADE615
:10077000B1E00D931C93A4E2B1E0E6E7F1E022279B
:1007800091E00E94E205002F003018F011F00C9467
:10079000CB030C94D203809169018F7B8093690114
:1007A0000C94D70380916901806480936901A4E26D
:1007B000B1E00E949308082F0F93A4E2B1E0E6E7AE
:1007C000F1E0222791E00E94E205402F0F91041BE7
:1007D000A3E7B1E00C93A4E2B1E00E949308EA2FF2
:1007E000FB2F009173013197E01BF10B0FEFA4E297
:1007F000B1E00E948B08A4E2B1E00E94A606EDE001
:10080000F0E0AFE6B1E00E948508EEECF1E10E9475
:10081000AF04AEE0B8E0ECE6F1E00E9409080E9407
:10082000A7040E94B604EEEDF1E10E94AF04AEE031
:10083000B8E0EDE6F1E00E94FA070E94A7040E94EA
:10084000B6040027A9E6B1E08C9186FB0EF401E026
:1008500040E0041711F00C943F04ECEEF1E10E942B
:10086000AF04AEE0B8E0EFE6F1E00E940D060E94B2
:10087000EA040E94A7040E94B6040C944504E4EF25
:10088000F1E10E94AF040E94B604089505D00E94D1
:10089000CD0500FC0CD008950024E89457FF02C059
:1008A00009D0689400F80BD010F80124089502D004
:1008B00009D00895509540954F5F5F4F0895E89493
:1008C00017FF0895009510950F5F1F4F68940895C6
:1008D000AEE0B8E018D0883091F08D3039F0332395
:1008E000C9F38D933A9563FE44D0F4CF63FC04C002
:1008F0008DE03FD08AE03DD088278C93089539D091
:1009000011973395E7CF0F929F93AF93BF937F9348
:100910008091A1008823E1F3F8948091A1008A9549
:100920008093A10090919F00A0E6B0E0A90F002461
:10093000B01D8C9193959F3309F4992790939F0054
:1009400078947F91BF91AF919F910F900895AEE001
:10095000B8E08D91882311F00CD0FBCF08950E9450
:10096000A206802D11F005D0FACF08958DE001D0B8
:100970008AE09F939FB79F93AF93BF930F937F930B
:100980009091E3009F33E1F3F8949091E300939505
:100990009093E30099270091E200A2EAB0E0A00F53
:1009A000B91F8C9303950F3309F400270093E200DD
:1009B000559A7F910F91BF91AF919F919FBF9F914A
:1009C00008953197F1F70895689462F80895E894CE
:1009D00062F808958DE207FD8D938F2D881F802F7B
:1009E000881F8F57082F6894F7F8802F87FF15C04E
:1009F00080958395082F80E38D938EE28D93802FD1
:100A0000815228F080E38D9399279C930895442781
:100A10000A95802F09F196D01FC0805230F09EE4D5
:100A20009D9381E48D939D93EFCF4427DF92EF92C6
:100A3000FF920F938FE1801B11F0082F83D089D094
:100A40009EE29D930F91FF90EF90DF9044270395D6
:100A5000003209F4D7CF2BD03F93E4EEFAE038E12F
:100A60002F2D1E2D0D2DFF24EE24DD244427000FF5
:100A7000111F221FA8F42F923F920E94A206102C51
:100A80000E94A206202C0E94A206302C0E94A206E0
:100A90003197410DD21CE31CF01C3F902F9001C0F8
:100AA000339631963A9519F73F9107D0AFCFDD0CC9
:100AB000EE1CFF1C0A95D9F70895002719E058D0BD
:100AC0008F93802B11F0039501C08F911A95B9F780
:100AD000802F882309F496CF8F91805D8D930A959E
:100AE000D9F792CF0065CD1D80B2E60E405973074D
:100AF000A0ACB90350D6DC01286BEE00943577002A
:100B0000CA9A3B0065CD1D00B2E60E00597307007E
:100B1000ACB90300D6DC01006BEE000035770000B5
:100B20009A3B0000CD1D0000E60E00007307000098
:100B3000B9030000DC010000EE00000077000000B7
:100B40003B000000F694E794D79447950A95D1F7B7
:100B5000089500270DD08F9303958F2D8E298D2911
:100B6000842BC1F78F91805D8D930A95D9F74CCF77
:100B70001F930F93002710E2440FDD1CEE1CFF1C97
:100B8000001F802F9AE0890B10F0082F43951A95CB
:100B900099F7802F0F911F9108950F92B801469FEA
:100BA0008001479F100D569F100D0F9008950E94D1
:100BB000A2060D920020D9F7089599910027A90F58
:100BC000B01F1197492F4A955E2F6F2FE894112778
:100BD0004395203019F0C895802D01C0808188236D
:100BE000B9F07C917723A1F0781739F40EF0042F37
:100BF0001395689411963196EBCF112321F0411B88
:100C0000A11B1127B10BE894E52FF62F1196E0CF29
:100C1000882311F0002708950895D190E190F19074
:100C20000191089521913191419151910895102F91
:100C300090E8FF0C001F0927990FF7941078652F93
:100C400090E8440F551F5927990F47956078003851
:100C50000895FF0C90E89027110F9795F794092FAE
:100C60000895502F2D2D3E2D4F2D612F08952DECE1
:100C70003CEC4CEC5DE366270FC0CFDFF2DFDD24F8
:100C8000EE2490E8F92E0FE307C0CCDF05C0222741
:100C9000332740E251E46627552351F1002381F1C7
:100CA000C6DF71F11627005850580894050B18F448
:100CB00007FD03C025C007FD23C04695379527953E
:100CC000F694E794D79422D0FF202AF0DD0CEE1C96
:100CD000FF1C015073F09D2D969548F0DD203AF4ED
:100CE000EE202AF491E0D90E9927E91EF91EB1CF22
:100CF00007C09FE7092FF92A9FEFD92EE92E089503
:100D0000DD24EE24FF240027112708959F929924C3
:100D1000AA24BB2488E1D216E306F40628F0D21AEE
:100D2000E30AF40A089401C08894991CAA1CBB1C0D
:100D3000DD0CEE1CFF1C8A9571F7D92CEA2CFB2CDC
:100D40009F900895C8953196002008950E94E70469
:100D5000E89488278A938A93D3DF11278D91803274
:100D6000E9F31197BBD098F08D3229F410951196C4
:100D70008C91B4D060F08E3229F411968C91AED063
:100D800008F446C022960E94E40481E008958C9104
:100D9000A5D0D8F547D01196D0F703958D919ED068
:100DA000E0F38E3229F48C9199D010F41196FBCF98
:100DB000853419F0853609F055C011968C918ED086
:100DC00060F08D3219F08B3221F0DCCF0880009476
:100DD000088211968C9182D0A8F68053898311964F
:100DE0008C917CD058F49981990F990F0980900DBE
:100DF000990F8053890F8983873220F689819881E2
:100E000099230AF48195080F2DC08E3289F6119628
:100E10008C9164D068F606D018F011960A95F8CF38
:100E20001196C1CF4F2D3E2D2D2DDD0CEE1CFF1C3C
:100E3000A8F0DD0CEE1CFF1C88F0D20EE31EF41EA1
:100E400068F0DD0CEE1CFF1C48F0805309F068943C
:100E5000D80E8827E81EF81E08F00895F42EE32E19
:100E6000D22E089534D019F116F5098308E921D05E
:100E70000695882787959F2D9F77980FF92E01500B
:100E8000000F110F07958981882379F01AF4819555
:100E9000898306C0ECDE89818A958983D9F705C0EC
:100EA000F6DE89818A958983D9F72296089528DF0D
:100EB000FCCF0DD041F0FF2032F00A9531F0DD0C6F
:100EC000EE1CFF1CD2F7889408950894089500241E
:100ED0000D280E280F28002A00200895803320F0C6
:100EE0008A3310F4089408958894089591E005C019
:100EF00092E003C094E001C098E024DF0D929A953F
:100F0000E1F70895819104D08D938823D9F708954E
:100F1000813618F08B3708F48F7D08957F930F93F7
:100F2000AF93BF938F939F938FB78F93E8948091E4
:100F3000A1000FE3081B21F49CB10E94E40413C03C
:100F40000091A000A0E6B0E077279CB1A00FB71FEA
:100F50009C93689483958093A10003950F3309F4C3
:100F600000270093A0009D3011F40E94A8018F91EA
:100F70008FBF9F918F91BF91AF910F917F911895E6
:100F80007F93AF93BF938F939F938FB78F939091DE
:100F9000E300992399F09A959093E3009927A2EAA8
:100FA000B0E08091E100A80FB91F9C9183958F3329
:100FB00009F488278093E1009CB901C055988F916E
:100FC0008FBF9F918F91BF91AF917F911895040F23
:100FD000151F261F371F0895000F111F221F331FD3
:100FE000089500951095209530950F5F1F4F2F4F56
:100FF0003F4F0895019110810EC0019111912191EF
:1010000030810BC00191108117FF05C03FEF2FEF1A
:1010100004C0008111272227332737FF03C0E1DFF7
:101020008DE28D93CF93DF93CF92DF92EF92AA243C
:10103000BB24CC24DD24EE2440E2CAE0DD2755E0C9
:1010400093E38881890F87FD9F7083FD907F891BC3
:1010500089935A95A9F7C0DFAA1CBB1CCC1CDD1CC8
:10106000EE1C4A9551F7E894EFE0FF2782910ED0ED
:10107000EB30E0F71EF068948A2D0CD088278D9312
:10108000EF90DF90CF90DF91CF910895982F8295C8
:1010900001D0892F8F70805D26F0803309F4089588
:1010A00068948D93089500271127222733271DD098
:1010B0008A3328F4803318F005D015D0F9CF0EF418
:1010C00090CF089580538F93402F512F622F732F0D
:1010D00083DF82DF7CDF80DF8F919927080F191F64
:1010E000291F391F08958D910895E894FCDF8032FF
:1010F000E9F38B32D9F38930C9F38D3211F4689456
:10110000F2CF089588278D93089594E081918D936F
:101110009A95E1F7089581918D930A9519F08823A6
:10112000D1F70895EFCF8FEF83959D919923E1F744
:101130000895689401C0E894AF93BF938D9116F021
:10114000919103C00E94A206902D891718F011F406
:101150008823A1F7BF91AF910895689463F808952B
:10116000000000003A003D00545247005354520022
:1011700049444E0056414C004F46530053434C00E7
:101180005241570050494F004449520044535000C7
:10119000414C4C004F50540054524D005452540096
:1011A00054524C00494342004943570049435300BD
:1011B00049435400494341005245460057454E00BB
:1011C00045524300534244004E4F50002A00234DE5
:1011D0006F64756C6E756D6D65723A2000002353F7
:1011E00075626368616E6E656C3A200023576572A4
:0611F000743A2000230008
:00000001FF
